:104B4C000000090101240200000301FA0400FA0527
:104B5C0000020A0A5A0B000F0C00FA0D00030E009B
:104B6C00030F0132100096120132130AFA140102DB
:104B7C0015000217010A18010A1905321A010A1B3D
:104B8C00010A1C053223011E2400642A00FA2B00A2
:104B9C00FA2C50782D003C2E00462F001E3000645D
:104BAC003250783300003432FA3501643601643700
:104BBC000150380A643C00643E003C3F000140FF59
:104BCC00FF411450420A5A430AC844053245007842
:104BDC004600FA4701234802034C00FA4EFFFF50EF
:104BEC000606510596520A32530B28540A96560162
:104BFC0002570546580002590A465A32FA5B010A16
:104C0C005C0A325E000A5F00FE61FFFF64021167FE
:104C1C0001036A0A3C6B00006C3296780132790110
:104C2C0032FAFAFA0000090101240200000301FA29
:104C3C000400FA0500020A0A5A0B000F0C00FA0DC8
:104C4C0000030E00030F0132100096120132130AFA
:104C5C00FA14010215000017010A18010A1905328D
:104C6C001A010A1B010A1C053223011E2400642AA6
:104C7C0000FA2B00FA2C50782D003C2E00462F0009
:104C8C001E3000643250783300003432FA3501643F
:104C9C00360164370150380A643C00643E003C3FE6
:104CAC00000140FFFF411450420A5A430AC8440510
:104CBC00324500784600FA4701234802024C00FABC
:104CCC004EFFFF500606510596520A32530B2854DC
:104CDC000A96560101570546580001590A465A32A0
:104CEC00FA5B010A5C0A325E000A5F00FE61FFFF9C
:104CFC006402116701036A0A3C6B00006C329678FF
:104D0C000132790132FAFAFA0065006F00790083FA
:104D1C00008D009700A100AC00B600C000CA00D402
:104D2C0000DE00E800F2005B0063006A0072007AAB
:104D3C00008200890091009900A100A800B000B881
:104D4C0000BF00C700CF00D600DF00E600EE00F683
:104D5C0000400046004C00520059005F0065006B9B
:104D6C0000710077007D00830089008F0095009C06
:104D7C0000A200A800AE00B400BA00C000C600CC6F
:0C4D8C0000D200D900DF00E500EB00F1D0
:10009E00AE33AF34740A8E048F05FF1250048C35C4
:1000AE008D36AE33AF34740A8E048F05FF12503D79
:1000BE008C338D34E53445336013740AC39534FFA5
:1000CE00E49533FE8E338F34783512507FE550A889
:1000DE0035B80015D395364010E550C39536FFE47C
:1000EE009535FE8E358F368010E5502424C3953617
:1000FE00FFE49535FE8E358F36AE35AF3674246FF0
:10010E004E700B7536237535007550018003755092
:10011E000022900084E0B40104C20B8002D20B9046
:10012E000085E0B40104C20C8002D20C9000C2E043
:10013E0075F0DCA4FFAEF0740A8E048F05FF12502A
:10014E00049007AAECF0A3EDF0A208401674038CFD
:10015E00068D0712502274011250149007A8EEF06B
:10016E00A3EFF07E017F00900080E01250229000FD
:10017E00C3E08E048F05FF125004740AFF12500460
:10018E008D399000CCE075F0DCA4FFAEF0740A8ED1
:10019E00048F05FF1250049007AEECF0A3EDF09023
:1001AE0000CEE060139000CEE0F5F0741684FF7E72
:1001BE0000EF9007B6F0800674649007B6F09000DA
:1001CE00D6E0B4020674029000B8F09000ADE0B430
:1001DE000B0874E390006FF080499000ADE0B41905
:1001EE00129000C3E0904CFF12008CE49390006FCD
:1001FE00F080309000ADE0B41E129000C3E0904D40
:10020E001D12008CE49390006FF080179000ADE00B
:10021E00B428109000C3E0904D4712008CE49390E8
:10022E00006FF090004BE0C39405502274019000D3
:10023E00C6F09000C8E0B4020674019000C8F090B9
:10024E0000B8E0D39402400674029000B8F090001B
:10025E00E0E0B40117900024740FF0A374FFF09047
:10026E000026E4F0A3F074029000E0F09000E0E0CD
:10027E00B40341900026E0FEA3E0FF900024E0FCD2
:10028E00A3E0FD125077741012502274081250140D
:10029E00EF90006CF0EF700674FF90006CF074003D
:1002AE009000E0F0900025E090006DF0900024E0CA
:1002BE0090006EF0900071E0900034F0900034E009
:1002CE00240C900035F0900034E02418900036F0A5
:1002DE00900035E0D39424400B900035E0C3942475
:1002EE00900035F0900036E0D39424400B90003609
:1002FE00E0C39424900036F090003AE4F09000347D
:10030E00E0B4240C90003A7401F09000347401F0C3
:10031E0090003BE4F0900035E0B4240C90003B7468
:10032E0001F09000357401F090003CE4F09000363E
:10033E00E0B4240C90003C7401F09000367401F08F
:10034E00900071E0FE9000D4E02E90003EF0900000
:10035E00AFE0B4014B90003EE06412600790003EA7
:10036E00E0B4240690003EE014F090003EE0D394FA
:10037E0024400B90003EE0C3942490003EF0900089
:10038E003EE0D39412400D90003EE0C394129000D4
:10039E003FF0800A90003EE0241290003FF080591A
:1003AE0090003EE0640C600F90003EE06418600721
:1003BE0090003EE0B4240690003EE014F090003E23
:1003CE00E0D39424400B90003EE0C3942490003E72
:1003DE00F090003EE0D3940C400B90003EE0C394AE
:1003EE000C90003EF090003EE0D3940C400B900039
:1003FE003EE0C3940C90003EF09000B7E0900037C2
:10040E00F0900037E0640C6007900037E0B41806F7
:10041E00900037E004F0900037E0240C900038F0A4
:10042E00900037E02418900039F0900038E0D39413
:10043E0024400B900038E0C39424900038F09000D4
:10044E0039E0D39424400B900039E0C394249000FB
:10045E0039F022C293C294C291C292C287C290E571
:10046E00B554EFF5B5E5B554DFF5B5C296C295C2F4
:10047E00A0C297C2A2C2A1E5B554BFF5B5E5B55469
:10048E007FF5B5E5B554FBF5B5C20D753746900051
:10049E00BAE07005754902800375490390000C742B
:1004AE00FFF0A374DCF090009BE0900012F8E4F0F3
:1004BE00E8A3F0C213C215C21774C8900028F074D6
:1004CE00C890002CF074C8900030F0752600752589
:1004DE0000C208756C00E54BB40903754B00753C02
:1004EE000090001AE4F0A3F0754C1E7528007527D5
:1004FE0000C210C211C2129007AAE0FEA3E0FF7460
:10050E000312502274011250149007A8EEF0A3EFBC
:10051E00F0C203900010E4F0A3F0C2222285F9503D
:10052E0085FA517E017F00E551125022E5502FFFD2
:10053E0050010E8E338F349007AAE0FCA3E0FDEF3E
:10054E002DFDEE3CFC8C358D36E536F5FBE535F5AF
:10055E00FC22053D22A2D8B34006C296C295C2A087
:10056E0075D8402285A74F75A7109000B8E0640398
:10057E0060079000D6E0B4022CA2D8B34002C2931A
:10058E00A2D9B34002C294A2DAB34002C291A2DB56
:10059E00B34002C292A2DCB34002C287A2DDB340D6
:1005AE0002C290801BA2D8B34004C293C292A2D9B9
:1005BE00B34004C294C287A2DAB34004C291C2907F
:1005CE0075D840854FA722900047E49364066002D9
:1005DE0080FE74C89007B0F8E4F0E8A3F075B5009B
:1005EE0075840175A70075FF8075EF0690003DE4D8
:1005FE00F075C91075A70F75A1C775A70075D9003D
:10060E0075CE0C75A70F75F1FE75F2FF75F30775B4
:10061E00F47875A4BA75A5FF75A60775AE0075AF0B
:10062E00FF75D48175D5FF75D6FF75D7FF75A700F9
:10063E0075A20175A14775F80975D80075D90475AD
:10064E00DA0975D84075A71075D80075D90475DA12
:10065E000975DB0975DC0975DD0975DE0975DF09BC
:10066E0075D84075A70075E60875E71075BC01755D
:10067E00BE0475BD6C75BE0775BDA075BE0875BD93
:10068E000175BC0075BB1875BC2075BA0875E8807D
:10069E0075D11375B50075A70F75E10575E2007577
:1006AE00C740C293C294C291C292C287C290E5B5AE
:1006BE0054EFF5B5E5B554DFF5B5C296C295C2A0B7
:1006CE00C297C2A2C2A1E5B554BFF5B5E5B5547F38
:1006DE00F5B5E5B554FBF5B5759700759780740AB9
:1006EE00124FF47597C0E5975420700280F8758FFD
:1006FE000275A700D2AF75980075A90C75A70F7576
:10070E00AB4375ADFB75AC1E75A71075C91875CAD0
:10071E000075CB0075C80475A700758912758E0417
:10072E00758C00758A00C2A9D28C758D00758B00F0
:10073E00D2ABD28E75D944753200753100752E004C
:10074E00752D00754600754700C29974C8F5097578
:10075E000800122F5875B50074639007B0F8E4F0D6
:10076E00E8A3F01231E47464F509750800122F58ED
:10077E00C21E90005AE0B40108A2B54002D21E80FB
:10078E002E90005AE0B4021175A70F75F30F75A7DE
:10079E0000A2A34002D21E801690005AE0B4030FAE
:1007AE0075A70F75F31775A700A2A44002D21EA25B
:1007BE001EB350030208AB74089007B0F8E4F0E8DB
:1007CE00A3F01230B37464F509750800122F587433
:1007DE00099007B0F8E4F0E8A3F01230B37464F5B2
:1007EE0009750800122F58740A9007B0F8E4F0E863
:1007FE00A3F01230B37464F509750800122F587403
:10080E000B9007B0F8E4F0E8A3F01230B37464F57F
:10081E0009750800122F58740C9007B0F8E4F0E830
:10082E00A3F01230B37464F509750800122F5874D2
:10083E000D9007B0F8E4F0E8A3F01230B37464F54D
:10084E0009750800122F58740E9007B0F8E4F0E8FE
:10085E00A3F01230B37464F509750800122F5874A2
:10086E00029000B9F090005AE090007DF090005A8E
:10087E00E0B401087400900085F0801C90005AE0EE
:10088E00B4020874009000C8F0800D90005AE0B4D5
:10089E00030674009000D5F0D21A02098B9007B0AF
:1008AE00E4F0A304F01230B37464F5097508001275
:1008BE002F5874029007B0F8E4F0E8A3F01230B3AA
:1008CE007464F509750800122F5874039007B0F878
:1008DE00E4F0E8A3F01230B37464F5097508001261
:1008EE002F5874049007B0F8E4F0E8A3F01230B378
:1008FE007464F509750800122F5874059007B0F846
:10090E00E4F0E8A3F01230B37464F5097508001230
:10091E002F5874069007B0F8E4F0E8A3F01230B345
:10092E007464F509750800122F5874079007B0F813
:10093E00E4F0E8A3F01230B37464F5097508001200
:10094E002F5874019000B9F090005AE090007DF09D
:10095E0090005AE0B401087400900085F0801C905D
:10096E00005AE0B4020874009000C8F0800D9000A8
:10097E005AE0B4030674009000D5F0C21A12335830
:10098E009000C3E07006740A9000C3F090006FE010
:10099E00700674E390006FF0120120E5B54401F586
:1009AE00B57406900049F0740190004AF0740390FB
:1009BE00004CF0740490004DF0740D90004EF074E5
:1009CE000590004FF090004BE0B4040674049000C4
:1009DE004FF07406900050F07400900055F07400C3
:1009EE00900056F07401900057F07400900058F08B
:1009FE0074FF900059F07433900147F074369001F3
:100A0E0048F0742D900149F0743190014AF0742031
:100A1E0090014BF0743390014CF0744390014DF003
:100A2E00747990014EF0746C90014FF07420900127
:100A3E0050F07420900151F07420900152F0742007
:100A4E00900153F07420900154F07420900155F0F1
:100A5E009000DFE090006CF0900096E090006DF05A
:100A6E00900097E090006EF0C213C215C21774C8C2
:100A7E00900028F074C890002CF074C8900030F0EC
:100A8E00C210C211C212A2B6B39209A2B3B3920A95
:100A9E00752600752500753746754C1E900068E466
:100AAE00F075271975286490000C74FFF0A374DCA0
:100ABE00F0C20D754B00C208752A00752900900012
:100ACE0010E4F0A3F0743A900770F074FD90077183
:100ADE00F0756D00900069E4F0752C00752B009098
:100AEE000014E4F0A3F090009BE0900012F8E4F004
:100AFE00E8A3F090007CE075F032A4FFAEF0900019
:100B0E0022EEF0A3EFF09007AAE0FEA3E0FF74033D
:100B1E0012502274011250149007A8EEF0A3EFF0B9
:100B2E00754A01900045E4F0C222C21F756C007533
:100B3E003C00C20EC20FC223C203754D00C204D2C6
:100B4E0005C206D207C21BC21CD21D74FE90004005
:100B5E00F074FE900041F0C220D221753800754429
:100B6E0000753A00753E32753F00754000743C903A
:100B7E000043F0754100743C900044F075420075DE
:100B8E00430090001AE4F0A3F0754500D2B2D2A44F
:100B9E00D2B0D2B1D2A3D2A7D2A6D2A5D2B790004C
:100BAE007CE0D394FA400674FA90007CF07E017FCC
:100BBE000090006EE012502290006DE02FFF500169
:100BCE000E900024EEF0A3EFF0EFD394FFEE940F0F
:100BDE004007900024E4F0A3F090006CE0700674DF
:100BEE00FF90006CF09000B9E0D3940240067401BF
:100BFE009000B9F09000BAE0700575490280037557
:100C0E0049039000BBE0D39401400674009000BBF2
:100C1E00F09000C1E0C3940A5006740A9000C1F02F
:100C2E009000CBE0700674019000CBF09000CBE00A
:100C3E00B4FF0674FE9000CBF09000D2E0D394FE89
:100C4E00400674FE9000D2F074019000D8F074014A
:100C5E009000D9F074009000DBF074009000E0F08A
:100C6E00D29CD2EC75CF01A298B35003021080C271
:100C7E0098E54764046006E59964FF6002802AA245
:100C8E00204004D2208020E547600874E625479076
:100C9E000045F0754700E546600874F02546900063
:100CAE0045F0754600C2208002C220E5476003026F
:100CBE000D5B754700E599B4FF03754601E599B4E0
:100CCE00FE03754602E599B4FD03754603E599B436
:100CDE00FC03754604E599B4FA03754605E599B427
:100CEE00FB03754701E599B4F903754704E599D3FC
:100CFE0094E54007E599C394F04002801685994823
:100D0E007547027E017F00E548C394E61250228E9D
:100D1E002F8F30753200753100E599D394C7400797
:100D2E00E599C394E64002801F8599487547037480
:100D3E00E5C39548F530752F00AE2FAF30904D9826
:100D4E00124FE3783112505DD299021080E547B40C
:100D5E0001028003020E33AE31AF3290007012509A
:100D6E0049E599F0783112507FAE31AF32EFB401D0
:100D7E0006EEB407028003020E33900770E0B43C17
:100D8E00028003020E1DC29C12046112012090000B
:100D9E006CE09000DFF090006DE0900096F0900017
:100DAE006EE0900097F0A21A4032755001E550D3D4
:100DBE0094075026E5509007B0F8E4F0E8A3F074DD
:100DCE00AA90003DF0122F847464F5097508001284
:100DDE002F587850740126F650D38030755008E5A0
:100DEE0050D3940E5026E5509007B0F8E4F0E8A3E7
:100DFE00F074AA90003DF0122F847464F509750802
:100E0E0000122F587850740126F650D312335874AE
:100E1E00C89007B0F8E4F0E8A3F0D29C75470075CF
:100E2E0046007599FBE547B402028003020EDDE52C
:100E3E00324531700685992E752D00AE31AF327464
:100E4E00016F4E701BAC2DAD2EAA2FAB30ED2BFBD0
:100E5E00EC3AFA8A068B07900070125049E599F029
:100E6E00783112507FAE31AF3274026F4E7060AC7B
:100E7E002DAD2E740D6D4C702C74639007B0F8E48C
:100E8E00F0E8A3F074AB90003DF090007DE0900090
:100E9E005AF01232BD90003DE4F074C89007B0F8DD
:100EAE00E4F0E8A3F0E548B4E619AE2DAF2E745683
:100EBE006F4E600C74486F4E600674666F4E700312
:100ECE00120461120120854899754700754600E5A8
:100EDE0047B4033FAE31AF32900070125049E599DE
:100EEE00F0783112507FAE31AF32AC2FAD308F0271
:100EFE008E038C068D07904DD4124FE3E493F97454
:100F0E000193FEEAD39EEB994009854899754700F7
:100F1E00754600E547B404028003021080AE31AF7F
:100F2E0032900070125049E599F0783112507FAE30
:100F3E0031AF32EFB40006EEB4010280030210802E
:100F4E00120461900053E075F002A4FFAEF08F50D2
:100F5E00EF900070125054EFFCE0FDEC9000731215
:100F6E005054EDFCE0FDEC2DFC900053E0B5040276
:100F7E0080030210710FEF900070125054E550FF75
:100F8E00E0FCEF900074125054ECFFE0FCEFC39CB9
:100F9E00FF900053E0B507028003021071E55090F8
:100FAE000072125054E550FFE0FCEF9000751250A5
:100FBE0054ECFFE0FCEF2CFF900053E0B5070280ED
:100FCE0003021071E550900076125054FFE0FCEFD2
:100FDE00900053E0F4042C90005AF0E55090007706
:100FEE00125054FFE0FCEF900053E0F4042C9000FC
:100FFE005BF0E550900078125054FFE0FCEF90004B
:10100E0053E0F4042C90005CF0E5509000791250FF
:10101E0054FFE0FCEF900053E0F4042C9007B0F87E
:10102E00E4F0E8A3F074AB90003DF01232BD7464AE
:10103E00F509750800122F589007B0125030123271
:10104E00BD7464F509750800122F589007B0125040
:10105E00301232BD7599F97464F509750800122FB6
:10106E005880FE7599FF7464F509750800122F58A3
:10107E0080FEE5466006A299B3B34003021200C299
:10108E0099E546B4011FAE31AF3290004912504976
:10109E00E0F599783112507FAE31AF3274116F4E48
:1010AE007003754600E546B40203854A99E546B4D9
:1010BE00031DAE31AF32900070125049E0F599EF3A
:1010CE00B40107EEB40703754600783112507FE580
:1010DE0046B4040280030211C2E532453170038525
:1010EE002699AE31AF3274016F4E7003853899AECA
:1010FE0031AF3274026F4E7003853A99AE31AF3212
:10110E0074036F4E7003853E99AE31AF3274046F27
:10111E004E7003854099AE31AF3274056F4E700339
:10112E00854199AE31AF3274066F4E700385429988
:10113E00AE31AF3274076F4E7003854399AE31AF47
:10114E003274086F4E700690001BE0F599AE31AF09
:10115E003274096F4E7017A221B340077599FAC207
:10116E0021800B900045E0F599900045E4F0AE31FA
:10117E00AF32740A6F4E7003854499AE31AF32743C
:10118E000B6F4E7003853F99AE31AF32740C6F4EBC
:10119E007003854599AE31AF32740D6F4E70037585
:1011AE0099FC783112507FAE31AF32740E6F4E70A3
:1011BE0003754600E546B4053990004BE0D3940420
:1011CE004010AE31AF32904B4C125049E493F5992A
:1011DE00800EAE31AF32904C30125049E493F599F7
:1011EE00AE31AF3274E36F4E700375460078311234
:1011FE00507FE54764016005E547B40403020C72B5
:10120E00C28E7E107F00E53D125022E58D75F010E6
:10121E00A4FDACF0EF2DFDEE3CFCE58B75F01084DB
:10122E00FF7E00ED2FFFEC3EFE8E278F28D28E9094
:10123E00009DE0605690001C12503090001CE0FCA7
:10124E00A3E0FD90001EE0FAA3E0FBEDB5033CEC3D
:10125E00B50238B219A208B34013A219B34008E57B
:10126E00B54404F5B58006E5B554FBF5B590001E02
:10127E00E0FEA3E0FF900020E0FCA3E0FDEF2DFDDB
:10128E00EE3CFC90001EECF0A3EDF09000AAE060A6
:10129E00099000AAE0C394034002807A124892A2F9
:1012AE0008B35009900068E0C3944640028006904F
:1012BE000094E0F56BE56B75F005A4FFAEF09007BA
:1012CE00B2EEF0A3EFF0900081E0C3953A4007E54F
:1012DE0038C3953950079007B2E4F0A3F0AE58AF7B
:1012EE00599007B2E0FCA3E0FDEFD39DEE9C4004C5
:1012FE00C2A1800B900068E0C394645002D2A1900A
:10130E0000AAE0B402099000B8E0C3940340028042
:10131E0005A2A1B392A29000AAE0B4031C1249AD9B
:10132E00AE58AF599007B2E0FCA3E0FDEFD39DEEAF
:10133E009C4004D2A18002C2A1900085E06009A267
:10134E00B3300A01B3B340028039A2B3300A01B3FD
:10135E004031A2B3300C01B3401C9000B8E0B4038E
:10136E0006A21BB3B3400280067405900045F0D26E
:10137E001BA20CB3920AA20CB330B301B34004A269
:10138E000C920AA2B6300901B35003021963A2B639
:10139E00300901B35003021963A2B6300B01B350EA
:1013AE000302187A754A0090009DE07013A20BB3E9
:1013BE004008E5B554FBF5B58006E5B54404F5B532
:1013CE000537A20DB3B35013AE27AF2890000CE033
:1013DE00FCA3E0FDEDC39FEC9E40030214E7E5493C
:1013EE00B40330E537B42405754901801FA222B33A
:1013FE00401AE537C3942450069000457401F0E579
:10140E0037D3942440067402900045F0753701D20C
:10141E0022805CE549B40206754901753724E5372B
:10142E00B424057537018047900045E07032E537EA
:10143E00C3942450069000457401F0E537D39424EC
:10144E0040067402900045F0E537C394245002D252
:10145E001FE537D394244002D21FC296C295C2A074
:10146E009000BAE0B402051204618003753701AE34
:10147E0029AF2AAC27AD28EF2DFDEE3CFC7403FFFF
:10148E001250048C298D2A90009DE0604390001C20
:10149E00E0FEA3E0FF90009DE08E048F05FF12504A
:1014AE000474018C068D07125014900020EEF0A3E8
:1014BE00EFF0900020E0F8A3E090001EC8F0A3C863
:1014CE00F090001CE4F0A3F0C219E5B554FBF5B59D
:1014DE00A21FB34002C21F802BAE29AF2AAC27AD8C
:1014EE0028EF2DFDEE3CFC74018C068D0712501476
:1014FE008E298F2AAC27AD28EDD39488EC94134017
:10150E0003120461E537B424127403900045F0D23F
:10151E001F9000BAE0B40203120461AE2BAF2CACE4
:10152E0027AD28EF2DFDEE3CFC8C2B8D2CAE27AF7E
:10153E0028EFD39DEE9C4011900014E0FAA3E0FB3F
:10154E00EBC394E8EA940340028006900014125014
:10155E0030900010E0FEA3E0FFAC27AD28EF2DFD8C
:10156E00EE3CFC900010ECF0A3EDF09000BAE0B46D
:10157E00021DAE27AF28740512502274038E048FFD
:10158E0005FF12500490000CECF0A3EDF08016AEA7
:10159E0027AF287403125022740112501490000CBD
:1015AE00EEF0A3EFF0C28E758D00758B00753D00C9
:1015BE00752801752700D28EE537240875F0098449
:1015CE00AFF07E00EF4E7075900010E0F8A3E09043
:1015DE00000EC8F0A3C8F090000EE0FEA3E0FFEFEF
:1015EE004E600B7C807D0E124F028E258F26900052
:1015FE0010E4F0A3F0AE25AF267428BE00039F5072
:10160E0010E53C2FFF50010E74011250148E258FE1
:10161E002685263C9000C1E0A825B8000DD395265E
:10162E004008E526900042F080099000C1E0149039
:10163E000042F0E54960067526007525009000B859
:10164E00E0B40308900037E0653760028026A21BE5
:10165E00B34004D21C8002B21C900085E0600BA245
:10166E001BB35006A21CB3B3400280067404900054
:10167E0045F0C21BE537640B6005E537B41D0990D4
:10168E0000AAE0600312459A9000AFE0B4011490F6
:10169E00003EE06537600790003FE0B53703754BBD
:1016AE0000801E90003EE06537601390003EE024FF
:1016BE000C6537600990003EE02418B53703754B72
:1016CE0000A20EB35006A20DB3B340030217CF9083
:1016DE000076E0B4015AE54075F00584FF7E009077
:1016EE000570125049E0F534753300AE33AF3490C7
:1016FE000074E012502274648E048F05FF125004A1
:10170E0074C18C068D071250228E358F36900012C2
:10171E00E0FEA3E0FFAC33AD3412000374648E041C
:10172E008F05FF125004900012ECF0A3EDF0800F25
:10173E00900074E075F0C1A4FFAEF08E358F36E5E3
:10174E003AC394CC5006900074E07002807175A775
:10175E001085F95085FA517E017F00E55112502215
:10176E00E5502FFF50010E8E338F34AC35AD36EF72
:10177E002DFDEE3CFC8C358D36D293D294D291E574
:10178E0036F5FBE535F5FCE536F5E9E535F5EAE543
:10179E0036F5EBE535F5EC9000B8E0B4031ED292C9
:1017AE00D287D290E536F5EDE535F5EEE536F5FD69
:1017BE00E535F5FEE536F5CEE535F5CF75A700D264
:1017CE000EE549B40106E537640B6002800F754CD7
:1017DE00019000487401F0E5B54401F5B5E54960A6
:1017EE00030218759000BDE0600D9000C4E0A825BE
:1017FE00B8000695264002803A9000BDE0B4021F64
:10180E00900034E06537600F900035E06537600773
:10181E00900036E0B53703754C03754500800CC259
:10182E000075450090001AE4F0A3F074099000458D
:10183E00F08034900034E0B5370B754C01900048C1
:10184E007401F08022900035E0B5370B754C0174B1
:10185E0002900048F08010900036E0B53709754CC4
:10186E00017403900048F0A20BB39209A20BB3309F
:10187E00B601B35003021963754A0190009DE070E2
:10188E0013A20BB34008E5B54404F5B58006E5B5E3
:10189E0054FBF5B5A20B9209E537D3944A4014D206
:1018AE000DE537D3946E400B7403900045F0D21FB4
:1018BE007537469000C5E0B40107E543C394144064
:1018CE000280031204617446900068F0A204300591
:1018DE0001B35017A204B34008E5B54408F5B5802E
:1018EE0006E5B554F7F5B5A2049205A20630070138
:1018FE00B35017A206B34008E5B54402F5B580060D
:10190E00E5B554FDF5B5A2069207E543C3944150E3
:10191E0009740E900045F012046190004FE0FE90A5
:10192E00004BE004C39E400990004BE0D394064068
:10193E000974FB900045F0120461900054E06015AC
:10194E00900054E0FE90004EE06E600974FE900030
:10195E0045F0120461A21FB34006C296C295C2A002
:10196E00A210B3B35008900037E065376003021A37
:10197E005CA202B35006A200B3B34003021A56751E
:10198E00A71085F95085FA517E017F00E55112505E
:10199E0022E5502FFF50010E8E338F34900018E049
:1019AE00FCA3E0FDEF2DFDEE3CFC8C358D3690005A
:1019BE00B8E0B4034EA208B34028A21CB3400CE515
:1019CE0036F5FBE535F5FCD293800AE536F5EDE507
:1019DE0035F5EED292A203B34004D2A28002C2A287
:1019EE00801FE536F5FBE535F5FCE536F5EDE5351D
:1019FE00F5EED293D292A203B34004D2A28002C2D9
:101A0E00A280429000D6E0C394025013E536F5FB57
:101A1E00E535F5FCD293A203B34002D2928026E5BF
:101A2E0036F5FBE535F5FCD293AE33AF34AC56AD9F
:101A3E0057EF2DFDEE3CFC8C358D36E536F5EDE59C
:101A4E0035F5EED29275A700C210D211D212A211A4
:101A5E00B3B35008900038E065376003021B4AA20A
:101A6E0002B35006A200B3B34003021B4475A71085
:101A7E0085F95085FA517E017F00E551125022E51D
:101A8E00502FFF50010E8E338F34900018E0FCA3C0
:101A9E00E0FDEF2DFDEE3CFC8C358D369000B8E070
:101AAE00B4034EA208B34028A21CB3400CE536F591
:101ABE00E9E535F5EAD294800AE536F5FDE535F52A
:101ACE00FED287A203B34004D2A28002C2A2801F1C
:101ADE00E536F5E9E535F5EAE536F5FDE535F5FEEC
:101AEE00D294D287A203B34004D2A28002C2A280B3
:101AFE00429000D6E0C394025013E536F5E9E53581
:101B0E00F5EAD294A203B34002D2878026E536F5D9
:101B1E00E9E535F5EAD294AE33AF34AC56AD57EFB6
:101B2E002DFDEE3CFC8C358D36E536F5FDE535F5B7
:101B3E00FED28775A700D210C211D212A212B3B371
:101B4E005008900039E065376003021C38A202B3DA
:101B5E005006A200B3B34003021C3275A71085F9DC
:101B6E005085FA517E017F00E551125022E5502F2B
:101B7E00FF50010E8E338F34900018E0FCA3E0FD71
:101B8E00EF2DFDEE3CFC8C358D369000B8E0B403A5
:101B9E004EA208B34028A21CB3400CE536F5EBE587
:101BAE0035F5ECD291800AE536F5CEE535F5CFD296
:101BBE0090A203B34004D2A28002C2A2801FE536D7
:101BCE00F5EBE535F5ECE536F5CEE535F5CFD2910D
:101BDE00D290A203B34004D2A28002C2A28042904D
:101BEE0000D6E0C394025013E536F5EBE535F5EC7F
:101BFE00D291A203B34002D2908026E536F5EBE5F2
:101C0E0035F5ECD291AE33AF34AC56AD57EF2DFD6A
:101C1E00EE3CFC8C358D36E536F5CEE535F5CFD27E
:101C2E009075A700D210D211C212E54CB40818124A
:101C3E003EC9A210B35005A211B340028006D210C5
:101C4E00D211D212754C1EE54CB40706123C8175AA
:101C5E004C08E54CB4063D900012E0FEA3E0FFEF09
:101C6E004E6006A208B3B340028023AE52AF53902B
:101C7E000012E0FCA3E0FDEF2DFDEE3CFC8C528D3E
:101C8E0053E537D3940C5006900012120039123AD5
:101C9E0053754C07E54CB405061238B3754C06E582
:101CAE004CB404329000ABE0902F3AF8282873120F
:101CBE0035478012123547800D1236F580081237DF
:061CCE00A780031237A7F6
:0F2F3A00021CBD021CC2021CC7021CCC021CD10F
:101CD40090008DE060051246838002C204754C05B5
:101CE400E54CB403028003021DCE900090E0600531
:101CF4001247908002C2069000ABE0D39402403FAA
:101D040090007FE02403A825B8000495265009908C
:101D14000081E0D3953A50028008D2027408900002
:101D240045F090007FE0A825B80005D39526500B18
:101D3400900081E02403C3953A5002C20280399096
:101D4400007FE02403A825B8000495265007E53851
:101D5400C3953940028008D2027408900045F0907F
:101D6400007FE0A825B80005D395265009E539245D
:101D74000FC395385002C2029000C5E07007E543D6
:101D8400C3941440028002D202A2024005754C049E
:101D9400800A754C1E90001AE4F0A3F0A208B34028
:101DA40029E54075F00584FF7E00900570125049C6
:101DB400E0C3946950051245CF800F9007AAE0F85C
:101DC400A3E09007A8C8F0A3C8F0E54CB40A0280C9
:101DD40003021E6C90002AE0C394465008C2967415
:101DE4004690002AF090003AE0B4011DE55A240A16
:101DF400F55A9007ACE0FEA3E0FF740A2FFF5001F0
:101E04000E9007ACEEF0A3EFF0855A3475330090D2
:101E14000034E0F55012009EE53690002AF0900060
:101E240006E533F0A3E534F0E55090002BF0C2143E
:101E34009007ACE0F533A3E0F534900034E0F550BE
:101E440012009EE536900028F0900000E533F0A3E0
:101E5400E534F0E550900029F0C213E549B40105DA
:101E6400754C0B8003754C03900028E0B53773A2C2
:101E740013404F900000E0FEA3E0FFEF4E6021AE60
:101E840029AF2A900000E0FCA3E0FD120003740ACD
:101E94008E048F05FF125004900000ECF0A3EDF0C7
:101EA400900029E0601A900000E0FEA3E0FFAC2956
:101EB400AD2AEF2DFDEE3CFC900000ECF0A3EDF01C
:101EC400D213AE27AF28900000E0FCA3E0FDEFC3DF
:101ED4009DEE9C400D12052BD296C21374C890003F
:101EE40028F0A213B3B35007900028E0B53702805E
:101EF4000D12052BD29674C8900028F0C2139000DE
:101F04002AE0B53770A214404F900006E0FEA3E02B
:101F1400FFEF4E6021AE29AF2A900006E0FCA3E05B
:101F2400FD120003740A8E048F05FF125004900002
:101F340006ECF0A3EDF090002BE0601A900006E0B0
:101F4400FEA3E0FFAC29AD2AEF2DFDEE3CFC900092
:101F540006ECF0A3EDF0D214AE27AF28900006E013
:101F6400FCA3E0FDEFC39DEE9C400AC2967446902C
:101F7400002AF0C214A214B3B3500790002AE0B5AB
:101F84003702800AC296744690002AF0C214E54CC7
:101F9400B40B02800302203B90002EE0C394465011
:101FA400139000C6E0B40104C2968002C295744640
:101FB40090002EF090003BE0B4011DE55A240AF590
:101FC4005A9007ACE0FEA3E0FF740A2FFF50010E05
:101FD4009007ACEEF0A3EFF0855A3475330090000F
:101FE40035E0F55012009EE53690002EF090000882
:101FF400E533F0A3E534F0E55090002FF0C21690DD
:1020040007ACE0F533A3E0F534900035E0F5501269
:10201400009EE53690002CF0900002E533F0A3E535
:1020240034F0E55090002DF0C215E549B401057572
:102034004C0C8003754C0390002CE0B5377EA21540
:10204400404F900002E0FEA3E0FFEF4E6021AE2976
:10205400AF2A900002E0FCA3E0FD120003740A8E94
:10206400048F05FF125004900002ECF0A3EDF090F1
:10207400002DE0601A900002E0FEA3E0FFAC29AD61
:102084002AEF2DFDEE3CFC900002ECF0A3EDF0D223
:1020940015AE27AF28900002E0FCA3E0FDEFC39D3E
:1020A400EE9C401812052B9000C6E0B40104D296B1
:1020B4008002D295C21574C890002CF0A215B3B357
:1020C400500790002CE0B53702801812052B9000C1
:1020D400C6E0B40104D2968002D29574C890002C54
:1020E400F0C21590002EE0B5377BA216404F900049
:1020F40008E0FEA3E0FFEF4E6021AE29AF2A900076
:1021040008E0FCA3E0FD120003740A8E048F05FFAF
:10211400125004900008ECF0A3EDF090002FE06062
:102124001A900008E0FEA3E0FFAC29AD2AEF2DFDD4
:10213400EE3CFC900008ECF0A3EDF0D216AE27AF15
:1021440028900008E0FCA3E0FDEFC39DEE9C401541
:102154009000C6E0B40104C2968002C29574469011
:10216400002EF0C216A216B3B3500790002EE0B5AD
:10217400370280159000C6E0B40104C2968002C202
:1021840095744690002EF0C216E54CB40C02800300
:10219400022234900032E0C3944650139000C6E00B
:1021A400B40104C2968002C2A07446900032F0903A
:1021B400003CE0B4011DE55A240AF55A9007ACE04E
:1021C400FEA3E0FF740A2FFF50010E9007ACEEF05F
:1021D400A3EFF0855A34753300900036E0F55012C1
:1021E400009EE536900032F090000AE533F0A3E556
:1021F40034F0E550900033F0C2189007ACE0F533AA
:10220400A3E0F534900036E0F55012009EE53690D8
:102214000030F0900004E533F0A3E534F0E550908D
:102224000031F0C217E549B40103754900754C0348
:10223400900030E0B5377EA217404F900004E0FED6
:10224400A3E0FFEF4E6021AE29AF2A900004E0FC2A
:10225400A3E0FD120003740A8E048F05FF125004DC
:10226400900004ECF0A3EDF0900031E0601A9000CF
:1022740004E0FEA3E0FFAC29AD2AEF2DFDEE3CFC0B
:10228400900004ECF0A3EDF0D217AE27AF28900035
:1022940004E0FCA3E0FDEFC39DEE9C401812052B67
:1022A4009000C6E0B40104D2968002D2A0C2177492
:1022B400C8900030F0A217B3B35007900030E0B5D7
:1022C4003702801812052B9000C6E0B40104D296A0
:1022D4008002D2A074C8900030F0C217900032E09F
:1022E400B5377BA218404F90000AE0FEA3E0FFEF51
:1022F4004E6021AE29AF2A90000AE0FCA3E0FD1253
:102304000003740A8E048F05FF12500490000AEC37
:10231400F0A3EDF0900033E0601A90000AE0FEA311
:10232400E0FFAC29AD2AEF2DFDEE3CFC90000AEC59
:10233400F0A3EDF0D218AE27AF2890000AE0FCA37A
:10234400E0FDEFC39DEE9C40159000C6E0B401048F
:10235400C2968002C2A07446900032F0C218A2183D
:10236400B3B35007900032E0B5370280159000C631
:10237400E0B40104C2968002C2A07446900032F018
:10238400C218E54CB402028003022436124332120E
:1023940044499007A8E0FEA3E0FF740A125022907B
:1023A400000EE0FCA3E0FD74098F02FF1250048DBF
:1023B400078C038E048A058B06124F029007ACEE3D
:1023C400F0A3EFF09000C6E0B401087450BE00051D
:1023D4009F4002800D74509007ACF8E4F0E8A3F03D
:1023E400801B9007ACE0FEA3E0FF74F0BE00039FE7
:1023F400500B74F09007ACF8E4F0E8A3F09007AC4D
:10240400E0FEA3E0FFE55A2FFF50010E9007ACEE6B
:10241400F0A3EFF0900048E0B40103754C0A90007B
:1024240048E0B40203754C0B900048E0B403037514
:102434004C0CE54CB401259000DDE0902F49F828C0
:1024440028731240D080121240D0800D12415A805D
:0924540008124206800312420640
:0F2F490002244602244B02245002245502245A2B
:10245D00754C029000C8E0B402028003022578900A
:10246D00006BE0D3953F506490006BE0F404253F82
:10247D00FE9000CBE08E00F5F0E884FF7E008F50DB
:10248D00EFC39410500CEF8550F0A4FDACF08D50BF
:10249D0080037550FF90006BE0D39550400B90007A
:1024AD006BE0C39550F54D8003754D009000E6E04F
:1024BD00D3954D40069000E6E0F54D9000E7E0C362
:1024CD00954D50069000E7E0F54D807190006BE062
:1024DD00C3953FFE9000CBE08E00F5F0E884FF7EC3
:1024ED00008F50EFC39410500CEF8550F0A4FDAC4D
:1024FD00F08D5080037550FF85503475330090007A
:10250D006BE02534FFAE3350010E8E338F3474FFE4
:10251D00BE0009D39F400585344D8003754DFF9056
:10252D0000E6E0D3954D40069000E6E0F54D9000B5
:10253D00E7E0C3954D50069000E7E0F54DA208B3D6
:10254D00B350099000D3E0D3954E5002800A740722
:10255D00900045F0C297801375A710E5CDC3954D3A
:10256D004004C2978002D29775A700E54BC394092A
:10257D004003022CB3A2EDB35003022CB3C2EDE520
:10258D004B6003022727900079E070030227169015
:10259D0000AFE0B40102800302267690003EE0B564
:1025AD00370280030226737E017F00E5BE125022A2
:1025BD00E5BD2FFF50010E8E338F34900079E0B4BE
:1025CD000118741012502290006FE08E048F05FFD9
:1025DD00125004ED900040F0802CAE33AF347410E7
:1025ED0012502290006FE08E048F05FF1250049060
:1025FD000040E02DFD50010C74018C068D0712502A
:10260D0014EF900040F0E54460089000D5E06402BE
:10261D00600280219000D7E0B4011A900040E0756F
:10262D00F0E7A4FFAEF0E5448E048F05FF125004D1
:10263D00ED900040F0900040E0FE900041E0D39E10
:10264D004004D21D8002B21D900040E0900041F088
:10265D009000ABE064016006A21DB3B3400280069A
:10266D00900040E0F538022714D21D7E017F00E571
:10267D00BE125022E5BD2FFF50010E8E338F3490C8
:10268D000079E0B40118741012502290006FE08EA2
:10269D00048F05FF125004ED900040F0802CAE33F6
:1026AD00AF34741012502290006FE08E048F05FF2E
:1026BD00125004900040E02DFD50010C74018C0669
:1026CD008D07125014EF900040F0E5446008900023
:1026DD00D5E06402600280219000D7E0B4011A9029
:1026ED000040E075F0E7A4FFAEF0E5448E048F05E1
:1026FD00FF125004ED900040F09000ABE0640160DB
:10270D0006900040E0F5388003753800900075E0C4
:10271D007005754B01800375BB18E54BB401028044
:10272D00030228C9900075E070030228B87E017F6E
:10273D0000E5BE125022E5BD2FFF50010E8E338FE6
:10274D00349000BBE0B4010F7E0F7FFFAC33AD348E
:10275D001250778E338F349000E0E0B40245AE33E3
:10276D00AF34900024E0FCA3E0FDEDD39FEC9E4040
:10277D000A900024E533F0A3E534F0AE33AF349086
:10278D000026E0FCA3E0FDEFD39DEE9C400A9000F7
:10279D0026E533F0A3E534F0AE33AF3474041250B4
:1027AD00148F3A9000E0E0704CAE33AF34900024BB
:1027BD00E0FCA3E0FDEFD39DEE9C40091250778E17
:1027CD00338F348006753400753300AE33AF3474F7
:1027DD001012502290006CE08E048F05FF125004F1
:1027ED008C338D347400D39D74019C400585343A2F
:1027FD008003753AFF9000ABE0B40102800302281C
:10280D00B6A208B3B3500E90007FE0A825B800051E
:10281D00D3952650030228AB900080E075F019A4E3
:10282D00FFAEF09000C3E08E048F05FF12500490B0
:10283D0000BCE0853AF0A4FFAEF074648D028C0309
:10284D008E048F05FF125004EA2DFDEB3CFC8C33FA
:10285D008D34E544600F9000D5E0B402089000D7A8
:10286D00E0640160028017AE33AF3474E71250227A
:10287D00E5448E048F05FF1250048C338D34900087
:10288D0040E0A833B8000AD395344005853438802C
:10289D000BA21DB34006900040E0F538800BA21D41
:1028AD00B34006900040E0F5388003753A00900083
:1028BD0078E07005754B02800375BB19E54BB402CA
:1028CD00028003022984900078E07003022973E5E9
:1028DD0037D3940C4003022971900022E0FEA3E04F
:1028ED00FFE53E12506F900022EEF0A3EFF07E0157
:1028FD007F00E5BE125022E5BD2FFF50010E8E3335
:10290D008F349000E5E07013740A12502274518ECA
:10291D00048F05FF1250048D3E8019AE33AF347411
:10292D000A1250228F048E057E017F95CDCCCD12DB
:10293D004F028F3EE53ED394644003753E64900094
:10294D0022E0FEA3E0FFE53E2FFF50010E90002296
:10295D00EEF0A3EFF090007CE0048E048F05FF12E3
:10296D0050048D3E8003753E329000C8E0700575B1
:10297D004B03800375BB13E54BB4035E9000C8E0B9
:10298D0060477E017F00E5BE125022E5BD2FFF504E
:10299D00010E8E338F3474041250148F3F9000CA81
:1029AD00E0853FF0A4FDACF07464FF1250048D3F40
:1029BD009000C9E0853FF0A4FFAEF074FF8E048F48
:1029CD0005FF1250048D4E8003753F00900076E098
:1029DD007005754B04800375BB17E54BB40402807D
:1029ED0003022A85900076E0B4017C7E017F00E52C
:1029FD00BE125022E5BD2FFF50010E74041250146B
:102A0D008E338F34900043E06012900043E01490B9
:102A1D004E1093A833B800069534400280069000FE
:102A2D0043E014F0900043E0C394775013900043BB
:102A3D00E004904E1093A833B80005D3953450029E
:102A4D008006900043E004F0900043E0FE90009C6F
:102A5D00E08E0088F0A4FFAEF074648E048F05FF45
:102A6D001250048D408003754000900077E0700592
:102A7D00754B05800375BB16E54BB405028003024B
:102A8D002B18900077E0B4017C7E017F00E5BE122B
:102A9D005022E5BD2FFF50010E74041250148E33D9
:102AAD008F34900044E06012900044E014904E8901
:102ABD0093A833B80006953440028006900044E098
:102ACD0014F0900044E0C394775013900044E00458
:102ADD00904E8993A833B80005D3953450028006E3
:102AED00900044E004F0900044E0FE9000A2E08EDF
:102AFD000088F0A4FFAEF074648E048F05FF1250B1
:102B0D00048D41800375410075BB1FE54BB4063341
:102B1D007E017F00E5BE125022E5BD2FFF50010E54
:102B2D008E338F34740912502274E68E048F05FF94
:102B3D001250048D4390007EE07005754B078003A5
:102B4D0075BB15E54BB407028003022C5A90007E2D
:102B5D00E07003022C497E017F00E5BE125022E594
:102B6D00BD2FFF50010E8E338F3474041250148F0D
:102B7D004290007EE0B401159000D2E08542F0A4B1
:102B8D00FFAEF07407125014EF9007B5F090007E71
:102B9D00E0B402159000D2E08542F0A4FFAEF074CF
:102BAD0007125014EF9007B4F090007EE0B40302CA
:102BBD008003022C479000BFE0701CE542C3940ACD
:102BCD005002D201E542D394644002C20190009EAE
:102BDD00E090006AF0806390009EE070349000D227
:102BED00E08542F0A4FFAEF074FF8E048F05FF1256
:102BFD005004ED90006AF0AE25AF26741EBE00069F
:102C0D00D39F4002D201E53AD394E54002C2018040
:102C1D0029E542C3940A500DAE25AF26741EBE00A1
:102C2D0004D39F50028002D201E53AD394E54002CD
:102C3D00C20190009EE090006AF080037542009002
:102C4D0000D5E07005754B08800375BB14E54BB4DA
:102C5D0008509000D5E060397E017F00E5BE12502E
:102C6D0022E5BD2FFF50010E8E338F34EFD394210B
:102C7D00EE940E40057544FF8015AE33AF347410DD
:102C8D0012502274E38E048F05FF1250048D448080
:102C9D0003754400900079E0600575BB1A800375DB
:102CAD00BB18054BD2ECAE27AF287410C39F742709
:102CBD009E400C900069E0C3943C4003022F37C244
:102CCD000D7537469000BAE07005754902800375A1
:102CDD004903C293C294C291C292C287C290E5B514
:102CED0054EFF5B5E5B554DFF5B5C296C295C2A062
:102CFD00C297C2A2C2A1E5B554BFF5B5E5B5547FE3
:102D0D00F5B5A21EB34008E5B54404F5B58006E55A
:102D1D00B554FBF5B5A20FB3500EE53AD39433403D
:102D2D0007E53AC394CC4003022DD5E5B54401F532
:102D3D00B57446900068F0900074E075F064A4FFDF
:102D4D00AEF08E358F367402BE000AD39F400675E5
:102D5D00360275350075A71085F95085FA517E013B
:102D6D007F00E551125022E5502FFF50010E8E339A
:102D7D008F34AC35AD36EF2DFDEE3CFC8C358D36FC
:102D8D00D293D294D291E536F5FBE535F5FCE536D7
:102D9D00F5E9E535F5EAE536F5EBE535F5EC9000C9
:102DAD00B8E0B4031ED292D287D290E536F5EDE5A8
:102DBD0035F5EEE536F5FDE535F5FEE536F5CEE511
:102DCD0035F5CF75A700D20FE53AC3941A5002C25C
:102DDD000F90000C74FFF0A374DCF090009BE0905A
:102DED000012F8E4F0E8A3F0C213C215C21774C8BC
:102DFD00900028F074C890002CF074C8900030F04A
:102E0D00C210C211C212752600752500753C00C294
:102E1D0008756C0090001AE4F0A3F0754C1E900735
:102E2D00AAE0FEA3E0FF74031250227401125014A5
:102E3D009007A8EEF0A3EFF090008DE0600512462C
:102E4D00838002C204900090E060051247908002DA
:102E5D00C206A204300501B35017A204B34008E521
:102E6D00B54408F5B58006E5B554F7F5B5A204925D
:102E7D0005A206300701B35017A206B34008E5B509
:102E8D004402F5B58006E5B554FDF5B5A2069207E9
:102E9D00C203752C00752B00900014E4F0A3F09084
:102EAD00007CE075F032A4FFAEF0900022EEF0A3AE
:102EBD00EFF0900010E4F0A3F0C222900069E0C39F
:102ECD00943C5010E54BB40909900069E004F0758D
:102EDD004B00803BE54BB40903754B00752800751D
:102EED002700758D00758B00753D00900068E0C35F
:102EFD0094645008900068E004F0800674649000BB
:102F0D0068F0900068E0B46406E5B554FEF5B59040
:102F1D000069E0D394014007E543C394414002802A
:0D2F2D0009740E900045F0120461020C7250
:104D98000000010001400160018001A001C001E0A4
:104DA80002000300039603B603D603F404000500CB
:104DB80005180530054805600578059005A805C063
:104DC800060006140628063C066E068C00FF013F06
:104DD800015F017F019F01BF01DF01FF02FF039512
:104DE80003B503D503F303FF04FF0517052F054794
:104DF800055F0577058F05A705BF05FF061306277D
:104E0800063B066F068B06A9DAD8D7D5D4D2D0CF01
:104E1800CDCBC9C7C6C4C2C0BEBCBAB8B5B3B1AFA2
:104E2800ADABA8A6A4A2A09D9B99969492908D8BB9
:104E380089878482807E7C79777573716F6D6B69E1
:104E4800676563615F5D5B5957565452504F4D4BD0
:104E58004A4847454442413F3E3C3B3A393736355C
:104E6800343231302F2E2D2C2B2A29282726252580
:104E78002423222121201F1E1E1D1C1C1B1A1A1947
:104E880019EEECEBEAE9E8E7E5E4E3E1E0DEDDDB97
:104E9800D9D8D6D4D2D0CECCCAC8C6C3C1BFBCBA62
:104EA800B7B5B2B0ADABA8A5A3A09D9B98959290BD
:104EB8008D8A8785827F7D7A7775726F6D6A68655E
:104EC80063615E5C5A575553514F4D4B49474543B3
:104ED80042403E3C3B393836353332312F2E2D2B6C
:104EE8002A292827262524232221201F1E1D1D1C90
:0A4EF8001B1A1A19181817161615C0
:102F5800750B00750A00AE0AAF0BAC08AD09EDC3DE
:102F68009FEC9E401674FF124FF475CF01780B74D6
:102F78000126F6500418E436F650DB2290003DE0B6
:102F8800B4AA1C900770E0B43C159007B0E0FEA30B
:102F9800E0FFEF4E6009741EBE0004D39F50030289
:102FA80030B275360075350075F8099007B0E0FE47
:102FB800A3E0FF74076F4E6006740E6F4E700674C0
:102FC8003A900770F09007B0E0FEA3E0FF7408BEE7
:102FD800001ED39F401A7E017F089007B0E0FCA333
:102FE800E0FD1DBDFF011C1200038E338F34801FCE
:102FF8009007B0E0FEA3E0FF740812506F8F048EB4
:10300800057E017F08CDCCCD1200038E338F34AE00
:1030180035AF36740CD39F74019E50030230ADA2B5
:10302800F9B3407EE5364535700375A382AE35AFFA
:103038003674016F4E700375A300AE35AF36740257
:103048006F4E700D9007B1E075F002A4FDACF08DE5
:10305800A3AE35AF3674036F4E700375A300AE355B
:10306800AF367403BE00039F5013AC33AD34ED2F5D
:10307800FFEC3EFE90006C125049E0F5A3AE35AF70
:1030880036EFB40B09EEB401057414124FF4AE35E3
:10309800AF36EFB40B07EEB4010375F80D783512AF
:1030A800507F02301790003DE4F0227536007535E8
:1030B8000075F8099007B0E0FEA3E0FF7408BE00B1
:1030C8001ED39F401A7E017F089007B0E0FCA3E062
:1030D800FD1DBDFF011C1200038E338F34801F902D
:1030E80007B0E0FEA3E0FF740812506F8F048E054E
:1030F8007E017F08CDCCCD1200038E338F34AE35E0
:10310800AF367411D39F74019E50030231E3A2F9C4
:10311800B350030231E0E5364535700375A3D2AEEE
:1031280035AF3674016F4E700375A300AE35AF36F8
:1031380074026F4E700D9007B1E075F002A4FDACFB
:10314800F08DA3AE35AF3674036F4E700375A300D0
:10315800AE35AF3674046F4E700375A300AE35AF4D
:103168003674056F4E700375A300AE35AF3674061E
:103178006F4E700375A300AE35AF3674076F4E708F
:103188000375A300AE35AF3674086F4E700375A390
:1031980000AE35AF367408BE00039F5016AC33AD91
:1031A80034ED2FFFEC3EFE900067125049E5A3F086
:1031B80075A300AE35AF36EFB41009EEB40105744F
:1031C80014124FF4AE35AF36EFB41007EEB4010366
:1031D80075F80D783512507F023106227536007564
:1031E800350075F809AE35AF367417BE0004D39FA5
:1031F80050030232BCA2F9B350030232B9E5364596
:1032080035700375A3D2AE35AF3674016F4E7003B7
:1032180075A300AE35AF3674026F4E700D9007B1CE
:10322800E075F002A4FDACF08DA3AE35AF367403A3
:103238006F4E700375A300AE35AF3674046F4E70D1
:103248000375A300AE35AF3674056F4E700375A3D2
:1032580000AE35AF3674066F4E700375A300AE35F9
:10326800AF3674076F4E700375A300AE35AF367472
:10327800086F4E700375A300AE35AF367408BE00F4
:10328800039F500C900051125049E5A3F075A3001C
:10329800AE35AF3674166F4E70057414124FF4AE17
:1032A80035AF3674166F4E700375F80D78351250B9
:1032B8007F0231ED2290003DE0B4AB02800302337F
:1032C8005775360075350075F809AE35AF36741286
:1032D800BE007CD39F4078A2F9B34070E5364535EF
:1032E800700375A382AE35AF3674016F4E700375E7
:1032F800A300AE35AF3674026F4E700D9007B1E083
:1033080075F002A4FDACF08DA3AE35AF3674036F33
:103318004E700375A300AE35AF367403BE00039F2D
:103328005009900056125049E0F5A3AE35AF3674F7
:10333800116F4E70057414124FF4AE35AF36741118
:103348006F4E700375F80D783512507F0232D22215
:10335800900046E4F074649007B0F8E4F0E8A3F055
:103368001231E474C89007B0F8E4F0E8A3F09000D4
:103378005DE0B4371A90005AE0900051F090005B7D
:10338800E0900052F090005CE0900053F08046908E
:1033980000467401F074659007B0F8E4F0E8A3F013
:1033A8001231E474C89007B0F8E4F0E8A3F0900094
:1033B8005DE0B4371A90005AE0900051F090005B3D
:1033C800E0900052F090005CE0900053F0800674AA
:1033D80002900046F0900047E4F074669007B0F859
:1033E800E4F0E8A3F01231E474C89007B0F8E4F010
:1033F800E8A3F090005CE0B4371290005AE0900027
:103408004BF090005BE0900054F080769000477499
:1034180001F074679007B0F8E4F0E8A3F01231E423
:1034280074C89007B0F8E4F0E8A3F090005CE0B44A
:10343800371290005AE090004BF090005BE090004B
:1034480054F0803E7402900047F074689007B0F81A
:10345800E4F0E8A3F01231E474C89007B0F8E4F09F
:10346800E8A3F090005CE0B4371290005AE09000B6
:103478004BF090005BE0900054F0800674039000DD
:1034880047F022E55D2534FFAE3350010E90007001
:10349800125049E0F55EE55D2534FFAE3350010E6C
:1034A8000FBF00010E900070125049E0F55F85656E
:1034B80061E55EB55F05855E5D8041E55FD3955E3C
:1034C800401DE55FC3955E8560F0A4FFAEF0E56141
:1034D8008E048F05FF125004ED255EF55D801DE515
:1034E8005EC3955F8560F0A4FFAEF0E5618E048F42
:1034F80005FF125004EDF404255EF55D22E55FD367
:10350800955E401DE55FC3955E8560F0A4FFAEF053
:10351800E5618E048F05FF125004ED255EF55D8090
:103528001DE55EC3955F8560F0A4FFAEF0E5618E92
:10353800048F05FF125004EDF404255EF55D22E5C5
:103548003875F00484FF7E008F5DE53875F00484DB
:10355800ADF07C008D60756504753301753400E548
:103568005DC3943F500512348B80069001AFE0F59F
:103578005D855D53755200900042E075F020A4FF10
:10358800AEF09000C1E08E048F05FF1250048D5DEF
:103598009000A9E0D39538500302364D9000CDE055
:1035A800D395384010ED9001B0125054E0F55575A0
:1035B800540002364A900098E0D395384043E55DC0
:1035C8009001B0125054E0F55EE55D9001D01250C4
:1035D80054E0F55F9000CDE0F4042538F5609000E4
:1035E80098E0FE9000CDE0F4042EF561E55EB55F4D
:1035F80005855E5D8003123505855D55755400802F
:1036080041E55D9001D0125054E0F55EE55D900112
:10361800F0125054E0F55F900098E0F4042538F576
:10362800609000A9E0FE900098E0F4042EF561E5B2
:103638005EB55F05855E5D8003123505855D557550
:1036480054000236F49000D0E0D395385011E55D6F
:10365800900230125054E0F5557554000236F4903B
:103668000099E0D395385043E55D9002101250540C
:10367800E0F55EE55D900230125054E0F55F900091
:1036880099E0F4042538F5609000D0E0FE900099A8
:10369800E0F4042EF561E55EB55F05855E5D8003A7
:1036A800123505855D557554008041E55D9001F042
:1036B800125054E0F55EE55D900210125054E0F5AA
:1036C8005F9000A9E0F4042538F560900099E0FEC9
:1036D8009000A9E0F4042EF561E55EB55F05855E0E
:1036E8005D8003123505855D55755400229000E113
:1036F800E0F562756511753302753400AE25AF26A5
:10370800E56275F00FA4FDACF0EDD39FEC9E40216F
:10371800E5628E048F05FF125004ED75F010A4FFCA
:10372800AEF0E53875F01184FD7C00ED2FF563806F
:103738000EE53875F01184FF7E00EF24F0F56385FF
:10374800635DE53875F01184AFF07E008F60123448
:103758008B855D64AE25AF269000E1E075F00FA47F
:10376800FDACF0EDD39FEC9E402875330275341004
:1037780085635D12348B85645E855D5FAE25AF26FB
:10378800E5628E048F05FF12503D8D6085626112DF
:103798003505855D53755200755564755400229042
:1037A80000E1E0F562756511753302753400AE25E8
:1037B800AF26E56275F00FA4FDACF0EDD39FEC9E4B
:1037C8004021E5628E048F05FF125004ED75F0105C
:1037D800A4FFAEF0E53A75F01184FD7C00ED2FF5FD
:1037E80063800EE53A75F01184FF7E00EF24F0F552
:1037F8006385635DE53A75F01184AFF07E008F60F4
:1038080012348B855D64AE25AF269000E1E075F03B
:103818000FA4FDACF0EDD39FEC9E402875330275E4
:10382800341085635D12348B85645E855D5FAE25DB
:10383800AF26E5628E048F05FF12503D8D608562CC
:1038480061123505855D537552009000ABE0B404F4
:1038580053E53875F00484FF7E008F5DE53875F018
:103868000484ADF07C008D60756504753301753492
:1038780000E55DC3943F500512348B80069001AF7C
:10388800E0F55DAE52AF53E55D12502274648E04CC
:103898008F05FF125004AE52AF53EF2DFDEE3CFCE6
:1038A8008C528D5375556475540022900076E0B49F
:1038B8000146E54075F00584FF7E008F5DE54075A3
:1038C800F00584ADF07C008D607565057533057570
:1038D8003400E55DC39417500512348B80069005BB
:1038E80087E0F55DAE54AF55E55D2FFF50010E74CE
:1038F8006412506F8E548F55900077E0B40146E5FE
:103908004175F00584FF7E008F5DE54175F0058403
:10391800ADF07C008D60756505753305753448E537
:103928005DC39417500512348B80069005CFE0F5DF
:103938005DAE54AF55E55D2FFF50010E7464125013
:103948006F8E548F55900086E0B40249E543C394C6
:103958004175F00584FF7E008F5DE54375F00584B1
:10396800ADF07C008D60756505753306753400E52E
:103978005DC39413500512348B8006900683E0F5DE
:103988005DAE54AF55E55D2FFF50010E74641250C3
:103998006F8E548F559000C8E0B402028003023A3B
:1039A80052E53875F01584FF7E008F5DE53875F0B7
:1039B8001584ADF07C008D6075651575330375341D
:1039C800F4E55DC3940B500512348B800690046FA8
:1039D800E0F55DE55D75F0FFA4FFAEF09000C9E08D
:1039E8008E048F05FF125004ED90006BF0E53F75D3
:1039F800F078A4FFAEF074FF8E048F05FF12500418
:103A08008C338D3474028C068D071250148F5DAC84
:103A180033AD347404FF12503D8D60756504753301
:103A28000675346EE55DC3941D500512348B80060F
:103A38009006FBE0F55DAE54AF55E55D2FFF5001F4
:103A48000E746412506F8E548F552290007EE0B42D
:103A580001179007B5E02555FFAE5450010E9000B0
:103A6800D2E012506F8E548F5590007EE0B403164A
:103A7800A201B3B3501090006AE0C39405A825B81A
:103A880000069526400280109000A0E02555FFAE64
:103A98005450010E8E548F55900078E0B402028085
:103AA80003023C8090007BE0602FE540D3941E40E9
:103AB80028900014E0FEA3E0FF9000B6E075F00344
:103AC800A4FDACF0EFD39DEE9C400E9000DAE0A888
:103AD80025B80005D395265003023C809000C3E02A
:103AE8008538F0A4FFAEF074051250227407125006
:103AF800148E338F34900082E0A825B800049526F0
:103B08005012900083E075F002A4FDACF0EFC39D65
:103B1800EE9C4003023C80E53875F00B84FF7E0084
:103B2800900600125049FEE0FFEE90007AE0FEEFAA
:103B38008E0088F0A4FFAEF074648E048F05FF1227
:103B480050048C338D34900042E075F018A4FFAE19
:103B5800F09000C1E08E048F05FF1250048C068D92
:103B680007900618125049AE33AF34E01250227451
:103B7800648E048F05FF1250048C338D34E53EA803
:103B880033B80077D395344072E53EC39534FFE4EB
:103B98009533FE8E338F347428BE00039F500C7506
:103BA8003428753300740D900045F0AE33AF34906F
:103BB800007BE012502274288E048F05FF125004F7
:103BC8008C338D34AE52AF53740A8E048F05FF12B6
:103BD80050048D068C07AC33AD34CFCECF12000322
:103BE800740A8E048F05FF1250048C338D34AE5244
:103BF800AF531250778E528F53807DE53EA833B86D
:103C0800000495345072AE33AF34E53E12506F8ED7
:103C1800338F347428BE00039F500C7534287533D5
:103C280000740D900045F0AE33AF3490007BE01285
:103C3800502274288E048F05FF1250048C338D3463
:103C4800AE52AF53740A8E048F05FF1250048D06CE
:103C58008C07AC33AD34CFCECF120003740A8E0478
:103C68008F05FF1250048C338D34AE52AF53EF2DB5
:103C7800FDEE3CFC8C528D5322AE52AF53AC54AD8A
:103C88005512000374648E048F05FF1250048C5281
:103C98008D53900073E08C068D0712502274648E49
:103CA800048F05FF1250048C528D53A2084017AEA2
:103CB80025AF267405BE00039F5002D208E53AD30B
:103CC80094CC4002D2029000D5E0B402089000D70C
:103CD800E0640160028017AE52AF53E544125022EF
:103CE80074E78E048F05FF1250048C528D53900098
:103CF80095E05402601B90008CE0A825B80012D310
:103D08009526400DA208B3B35007E53AC3949A40EC
:103D1800028028AE5BAF5C90008AE075F002A4FDDB
:103D2800ACF0EF2DFDEE3CFC74022DFD50010CE5CE
:103D38003ABC0007D39D4003756901853A5C755B01
:103D480000E5697003023DD79000E8E0C39569403B
:103D580070E54075F00584FF7E00900570125049AB
:103D6800E0F534753300AE33AF3490009AE012506A
:103D78002274648E048F05FF1250048C358D3690A2
:103D880000E8E004C395698C068D07125022900064
:103D9800E8E08E048F05FF1250048C358D369000B4
:103DA8008BE08C068D07125022740A8E048F05FF53
:103DB800125004AE52AF53EF2DFDEE3CFC8C528DE9
:103DC8005305699000E8E0C3956950037569009050
:103DD8000095E05401601B900089E0A825B8001206
:103DE800D39526400DA208B3B35007E538C394CC49
:103DF80040028025900087E075F003A4FFAEF0E54F
:103E0800662FFF50010E74032FFF50010EE538BED8
:103E18000007D39F4003756A01853866E56A700319
:103E2800023EB29000E9E0C3956A4070E54075F043
:103E38000584FF7E00900570125049E0F534753313
:103E480000AE33AF3490009AE012502274648E04AE
:103E58008F05FF1250048C358D369000E9E004C3BD
:103E6800956A8C068D071250229000E9E08E048F27
:103E780005FF1250048C358D36900088E08C068D35
:103E880007125022740A8E048F05FF125004AE5296
:103E9800AF53EF2DFDEE3CFC8C528D53056A90001C
:103EA800E9E0C3956A5003756A0090009AE0A85249
:103EB800B800049553500990009AE0F553755200E4
:103EC800229000D6E0B401028003023FD4A208B3D6
:103ED8005003023FD29000A1E0B40168AE52AF5344
:103EE800AC25AD26120003743C8E048F05FF1250DA
:103EF800049000B1E0BC00109D400D9000B3E0A814
:103F080052B8000495535002D203AE52AF53AC25B9
:103F1800AD26120003743C8E048F05FF12500490E6
:103F280000B1E0C3940ABC0015D39D40119000B3C2
:103F3800E0C39405A852B80005D3955350028002F7
:103F4800C2038068AE52AF53AC25AD26120003748D
:103F5800788E048F05FF1250049000B1E0BC001069
:103F68009D400D9000B3E0A852B80004955350044A
:103F7800D2038038AE52AF53AC25AD26120003747D
:103F8800788E048F05FF1250049000B1E0C3940AA4
:103F9800BC0015D39D40119000B3E0C39405A8520E
:103FA800B80005D3955350028002C203A203B34060
:103FB80019AE52AF539000B2E012502274648E04CE
:103FC8008F05FF1250048C528D538002C20390005B
:103FD800D6E0B40258E53875F00884FF7E008F5D9E
:103FE800E53875F00884ADF07C008D60756508755E
:103FF80033017534E0E55DC3943F500512348B807E
:104008000690026FE0F55DE55D75F05EA4FFAEF029
:10401800740A8E048F05FF1250048C568D57740253
:10402800BC000AD39D4006755702755600A200B31E
:104038004006A202B3B3500990001AE4F0A3F0803E
:1040480024AE52AF537400D39F74019E400C90006D
:104058001AE552F0A3E553F0800B74FF90001AF8AC
:10406800E4F0E8A3F09000B8E0D394024006A20878
:10407800B3B34002800DAE52AF5374021250228E79
:10408800528F539000A1E0B4010DAE52AF537402A9
:104098001250228E528F53AE52AF53745E1250227A
:1040A800740A8E048F05FF1250048C528D537402CB
:1040B800BC000AD39D400675530275520090001843
:1040C800E552F0A3E553F022900042E0900370120D
:1040D8005054E0F567756864900042E0FE9000ACCB
:1040E800E0D39E4037E53875F00884FF7E008F5D89
:1040F800E53875F00884ADF07C008D60756508754D
:104108003303753496E55DC3941F500512348B80D4
:1041180006900425E0F55D855D688035E53875F025
:104128000884FF7E008F5DE53875F00884ADF07C6B
:10413800008D607565087533037534B6E55DC39405
:104148001F500512348B8006900445E0F55D855DAF
:1041580068229000E2E0F5627565117533047534E4
:1041680000AE25AF26E56275F00FA4FDACF0EDD3E7
:104178009FEC9E4021E5628E048F05FF125004EDEE
:1041880075F010A4FFAEF0E53875F01184FD7C00E1
:10419800ED2FF563800EE53875F01184FF7E00EF92
:1041A80024F0F56385635DE53875F01184AFF07E22
:1041B800008F6012348B855D64AE25AF269000E2D7
:1041C800E075F00FA4FDACF0EDD39FEC9E40287590
:1041D800330475341085635D12348B85645E855DA8
:1041E8005FAE25AF26E5628E048F05FF12503D8D28
:1041F80060856261123505855D6775686422900087
:10420800E2E0F562756511753304753400AE25AFCB
:1042180026E56275F00FA4FDACF0EDD39FEC9E404F
:1042280021E5628E048F05FF125004ED75F010A48D
:10423800FFAEF0E53A75F01184FD7C00ED2FF563D3
:10424800800EE53A75F01184FF7E00EF24F0F563E7
:1042580085635DE53A75F01184AFF07E008F6012DA
:10426800348B855D64AE25AF269000E2E075F00FD3
:10427800A4FDACF0EDD39FEC9E4028753304753453
:104288001085635D12348B85645E855D5FAE25AFF6
:1042980026E5628E048F05FF12503D8D60856261B0
:1042A800123505855D677568649000DDE0B40479B2
:1042B800900042E0FE9000ACE0D39E4037E53875B0
:1042C800F00884FF7E008F5DE53875F00884ADF056
:1042D8007C008D60756508753303753496E55DC39C
:1042E800941F500512348B8006900425E0F55D85F7
:1042F8005D688035E53875F00884FF7E008F5DE5E0
:104308003875F00884ADF07C008D607565087533EC
:10431800037534B6E55DC3941F500512348B8006CF
:10432800900445E0F55D855D6822900076E0B40173
:104338003BE54075F00584FF7E008F5DE54075F034
:104348000584ADF07C008D607565057533057534A1
:1043580018E55DC39417500512348B800690059FAD
:10436800E0F55DE568255DC39464F568900077E045
:10437800B4013BE54175F00584FF7E008F5DE541A2
:1043880075F00584ADF07C008D60756505753305A5
:10439800753460E55DC39417500512348B80069020
:1043A80005E7E0F55DE568255DC39464F568E567B4
:1043B8002568F55A90007EE0B402109007B4E02515
:1043C8005AFE9000D2E0F4042EF55A9000D5E0D3BE
:1043D80094014040E544C394E7501D74E7C39544F5
:1043E800FE9007B6E08E00F5F0E884FF7E008F5D52
:1043F800E55A255DF55A801CE544C394E7FE90070D
:10440800B6E08E00F5F0E884FF7E008F5DE55AC3C4
:10441800955DF55AA2084006E5672464F55AE55A01
:10442800D394644009E55AC39464F55A8003755AD5
:10443800009000AEE0C3955A50069000AEE0F55AE1
:1044480022D2009000C4E0A825B800049526503B6D
:104458009000C4E0A825B8000495265003755A0FAB
:104468009000C4E004A825B8000495265003755AA6
:104478000A9000C4E02402A825B800049526500537
:10448800755A05C2007409900045F07E017F0090BE
:1044980000B4E01250229000C3E08E048F05FF1292
:1044A8005004E538BC000CD39D4008C200740A9043
:1044B8000045F09000B5E0C39540500D9000C7E06E
:1044C800A825B80006952640028008C200740B9003
:1044D8000045F0A2004003755A0590007EE0B40341
:1044E80006A201B3B34002802B90006AE0C3940592
:1044F800A825B800049526500C90009FE0F55A7442
:104508000C900045F090006AE0A825B800049526B4
:104518005002C200855A45900070E0255AFE90006E
:1045280042E075F01E84FC7F00EE2CF55A229000C4
:1045380042E075F00584FF7E008F5D900042E075D3
:10454800F00584ADF07C008D6075650575330375E5
:1045580034D69000C1E01475F00584FF7E00E55D57
:10456800BE00039F500512348B800BE55D90044616
:10457800125054E0F55DE55D9007B7F09007B7E09D
:10458800FE9000B0E0C39E50089000B0E09007B7DE
:10459800F022E54075F00584FF7E0090057012500A
:1045A80049E0F56CE56CD394644010E56CC3946401
:1045B80075F00F84FF7E008F6C8003756C0090008F
:1045C80093E0256CF56C229007AAE0FEA3E0FF7447
:1045D80004125014E538125022740F8E048F05FF10
:1045E8001250049007A8ECF0A3EDF0900086E0B418
:1045F8000262E543C3944175F00584FF7E008F5D38
:10460800E54375F00584ADF07C008D607565057532
:104618003306753414E55DC39417500512348B8046
:1046280006900697E0F55D9007A8E0FEA3E0FF740A
:104638000A8E048F05FF125004E55D8C068D071263
:104648005022740A8E048F05FF1250049007A8ECBC
:10465800F0A3EDF09007A8E0FEA3E0FF9007AEE01E
:10466800FCA3E0FDEDD39FEC9E400F9007AEE0F871
:10467800A3E09007A8C8F0A3C8F02290008DE0B48A
:10468800010385265090008DE0B402129000C3E02B
:104698008538F0A4FFAEF074081250148F509000C3
:1046A8008DE0B40303853A5090008DE0B40403858F
:1046B800405090008DE0B4050385415090008DE096
:1046C800B4060385425090008DE0B407038543503B
:1046D80090008DE0B4080385445090008DE0B40943
:1046E80003853F5090008DE0B40A03853E5090004A
:1046F8008DE0B40B0385455090008DE0B40C069016
:10470800001BE0F55090008EE0FE90008FE0D39EF5
:10471800404B90008DE0B4041890008FE0C3955092
:104728005002D20490008EE0D395504002C204801B
:104738002A90008EE0C39550500990008FE0D395E1
:104748005050028002D20490008EE0D39550500958
:1047580090008FE0C395505002C204802A90008ECA
:10476800E0D39550400990008FE0C39550400280F7
:1047780002C20490008EE0C39550400990008FE07B
:10478800D395504002D20422900090E0B4010385F2
:104798002650900090E0B402129000C3E08538F0F3
:1047A800A4FFAEF074081250148F50900090E0B43B
:1047B8000303853A50900090E0B40403854050907C
:1047C8000090E0B40503854150900090E0B40603E2
:1047D800854250900090E0B40703854350900090C4
:1047E800E0B40803854450900090E0B40903853F85
:1047F80050900090E0B40A03853E50900090E0B4D9
:104808000B03854550900090E0B40C0690001BE027
:10481800F550900091E0FE900092E0D39E404090C9
:104828000091E0C395505009900092E0D395505004
:10483800028002D206900091E0D395505009900072
:1048480092E0C395505002C206900090E0B401096E
:104858009000CFE0D3953A50028002C206802A9099
:104868000091E0D395504009900092E0C3955040E4
:10487800028002C206900091E0C395504009900062
:1048880092E0D395504002D20622AE58AF5974F543
:10489800D39F74019E4008785812507F0249AC7526
:1048A8005901755800AE25AF26E56CBE000DD39FA3
:1048B80040099000A5E0D3956D40028023756D00F6
:1048C800E56CC39526F5509000A8E0D3956B400899
:1048D800E56B2550F56B80069000A8E0F56B80022B
:1048E800056D900081E0D3953A401CE538C39539B1
:1048F8004015AE25AF26E56CBE00039F5009900019
:10490800A6E0D3956E4002806E9007B8E0A825B85F
:104918000004952650037570009007B8E0A825B8E4
:10492800000BD395264006E5269007B8F0E5707091
:1049380041E526C3956CF550E550D39405400375C1
:1049480050059000A7E0C3956B5007E550C3956BE1
:1049580040028009E56BC39550F56B80069000A76F
:10496800E0F56B9000A7E0D3956B40069000A7E0B8
:10497800F56B756E008002056EE57070169000810B
:10498800E0C3953A500DE56C2405A825B8000695B6
:10499800264002800F900094E0F56B7570017478E2
:1049A8009007B8F022AE58AF5974E9D39F74039EAC
:1049B8004008785812507F024B4B755901755800C2
:1049C800756B32A223402A756B19900094E075F03C
:1049D80002A4FFAEF0E56DBE0006D39F4002D223CD
:1049E800056D75700374789007B8F0756F00024B09
:1049F8003AAE25AF26E56C6F4E7003024B3AE56C74
:104A0800BE000DD39F40099000A5E0D3956D4002EC
:104A1800800F756D00E570C394035003756B1980A2
:104A28000DE56CC39526F550E56D2550F56D9000A4
:104A380081E0D3953A400E9007B8E0A825B8000762
:104A4800D395264002800C056F900094E0B56F0363
:104A5800757000E570B40306A208B3B34002800A7B
:104A6800056FE56FB43C03757002E570B4022990D8
:104A780007B8E0A825B8000ED395264009E526908A
:104A880007B8F0756F00900081E0C3953A5009753A
:104A98006F0074789007B8F0E570705A900081E064
:104AA800D3953A401CE538D395394015AE25AF2645
:104AB800E56CBE00039F50099000A6E0D3956E40B8
:104AC800028008756E00756B4B8028E526C3956CCF
:104AD800F550E550D394054003755005900081E0EA
:104AE800D3953A4008E56E2550F56E8006E56E24AC
:104AF80006F56E756F00E5707016900081E0C3953D
:104B08003A500DE56C2405A825B800069526400204
:104B18008003757001E570B40118756B19056F9005
:104B28000094E0B56F06757002756F007478900791
:104B3800B8F0E56B75F00AA4FFAEF09007B2EEF09E
:044B4800A3EFF022C5
:095054002582F582500205832239
:0F008C0025E050020583258250020583F582226C
:104FE300EF2F500205832582F582E5833E2EF5835C
:014FF300229B
:10506F00CFC39FFF50011E22C3EF9DFFEE9CFE2278
:09505D00E493F608740193F622B5
:08507F000806B6000218062223
:0D503000A3E004F07006120049E004F02235
:0E003900A3E014F0B4FF06120049E014F02218
:0E501400048007C3CE13CECF13CFD5E0F62213
:104F0200BC000FBE0008ED8FF084FFADF022E4FE7E
:104F1200FF22BE000DEF60FE54F0606F20E7030237
:104F22004FB8EAC0E0EBC0E078017A0075F001EE1C
:104F320020E710EF25E0FFEE33FE0AC5F023C5F0AF
:104F420030E7F0EA5407F9096A7A007B0060010849
:104F5200C3EC9E40167004ED9F4010ED9FFDEC9E49
:104F6200FCE5F0CA4ACA03F5F08005E5F003F5F066
:104F7200C3EE13FEEF13FFD9D77908CACBCAD8D034
:104F8200EAFEEBFFD0E0FBD0E0FA22EC8FF084FCEB
:104F9200ED54F045F0C48FF084FEEDC454F045F0BA
:104FA200C48FF084FDEEC4FE54F02DFFEE540F3C8E
:104FB200FEADF07C0022790078008FF0EC7E0820B4
:104FC200E70DC3CD33CD33C933C9C833C8DEF0844E
:104FD20049F9E5F08FF0BE00E6FD7C00E9FFE8FE4E
:014FE20022AC
:0E502200F88FF0A4FFE5F0CE88F0A42EFE2259
:10000300EF8DF0A4F9A8F0EF8CF0A428F8EE8DF0B2
:06001300A428FEE9FF2213
:104FF400600D782B024FFE007830D8FED5E0F82201
:10500400EEC0E07E00124F02EFFDEEFCD0E0FE2287
:0C503D00EEC0E07E00124F02D0E0FE2228
:03001B0002001EC2
:0300530002005652
:03009B00020071EF
:0300000002506645
:0950660075817175D0000205D5B9
:0B504900E5822FF582E5833EF583220F
:0A0049000582D5820215831582227C
:10001E00C0E0C0F0C083C082C0D075D000120560B1
:0B002E00D0D0D082D083D0F0D0E032E0
:10005600C0E0C0F0C083C082C0D075D00012056376
:10006600D0D0D082D083D0F0D0E032C0E0C0F0C093
:1000760083C082C0D075D000120572D0D0D082D095
:0600860083D0F0D0E0324F
:00000001FF
